:020000040000FA
:020000000528D1
:0800080009008316FF3085009A
:1000100086011130870006309F0040309400831223
:10002000003094009416850186010717B520303002
:100030008F20972007302D060319192806302D062A
:10004000031D8628972007302D06031D222807133D
:10005000813011210717A120AE0803192B28B130D8
:100060002E06031D742820308F20972007302D0680
:100070000319352805302D06031D862897200730E3
:100080002D06031D3E280713823011210717A120DA
:10009000AE0803194728B2302E06031D742810300D
:1000A0008F20972007302D060319512803302D0685
:1000B000031D8628972007302D06031D5A28071395
:1000C000843011210717A120AE0803196328B3302B
:1000D0002E06031D742830308F2064301A21003022
:1000E0008F20FA301A216B2820308F20FA301A2105
:1000F00030308F20FA301A21742810308F20FA30D7
:100100001A2130308F20FA301A217D2810308F20AC
:10011000FA301A2120308F20FA301A2186283039FF
:10012000AD000C30AB003030AC00062108000D30C3
:10013000AB00F3203830AD050310AD0CAD0CAD0CA9
:100140000800AE01FE20A01C080001301A212C304E
:10015000AB000230AC000301AD00062101301A21D2
:100160007130AB00F320AE000800E4208030D120D5
:100170008030A50007130230112100301121A701A2
:1001800045302707A80001300318013E8A002808DF
:1001900044211121A70AA50BC02807170030D12040
:1001A0000800A6000F30AB002608AD00EA200130A1
:1001B0001A210E30AB00F320E0302D052606031D7A
:1001C000D22801301A2108000713C0301121071767
:1001D0003F2108000713023011212B0811212D089F
:1001E0001121071708000713033011212B081121D3
:1001F0005A30112107172008AD0008000713A0305E
:1002000011215A3011210717200808000713053063
:1002100011212B0811212C0811212D08112107175C
:100220000800A10093008316141C142983121308DC
:10023000A0000800A300F630A200000000000000AB
:1002400000000000000000000000000000000000AE
:10025000000000000000000000000000A20B1D29AB
:10026000A30B1B290800A400FA301A21FA301A2126
:10027000FA301A21FA301A21A40B342908000A3066
:10028000A200A20B412908008200FF34FF34FF3492
:10029000FF34FF34FF34FF34FF34B1340034FF3413
:1002A000FF340C34003480348034B2340034FF34F2
:1002B000FF34B3340034FF34FF34FF34FF34FF34F1
:1002C000FF340034003480348034FF34FF34FF3492
:1002D000FF34FF34E034FF34FF3402349034093407
:1002E000033400340034803480340334C1340034A7
:1002F000003400340034003400340034003400345E
:10030000003400340034803480340234C234003489
:10031000003400340034003400340034003400343D
:10032000003400340034803480340134C334003469
:10033000003400340034003400340034003400341D
:1003400000340034003480348034203400340034ED
:1003500000340034003400340034003400340034FD
:1003600000340034003480348034203400340034CD
:1003700000340034003400340034003400340034DD
:0A038000003400340034803480346F
:02400E003A3F37
:00000001FF
